:100000000C9477000C946B020C946B020C946B02B2
:100010000C946B020C946B020C946B020C946B02AC
:100020000C946B020C946B020C946B020C946B029C
:100030000C946B020C946B020C946B020C946B028C
:100040000C946B020C946B020C946B020C946B027C
:100050000C946B020C946B020C946B020C946B026C
:100060000C946B020C946B020C946B020C946B025C
:100070000C946B020C946B020C946B020C94FA00BF
:100080000C946B020C946B020C946B020C946B023C
:100090000C946B020C946B020C946B020C946B022C
:1000A0000C946B020C946B020C946B020C946B021C
:1000B0000C946B020C946B020C946B020C946B020C
:1000C0000C946B020C946B020C946B020C946B02FC
:1000D0000C946B020C946B020C946B020C946B02EC
:1000E0000C946B020C946B02400040848000809161
:1000F00001108F7C806080688093011011241FBEE6
:10010000CFEFCDBFDFE7DEBFE8EEF0E040E019C0A3
:10011000B791A79137912791079107FD0EC097914D
:100120008791EF01F92FE82F0BBF07900D92A217CF
:10013000B307D9F7FE011BBE04C01D92A217B30777
:10014000E1F7ED3EF40721F70E9401020C943E0214
:04015000F894FFCF51
:100154005B4C4F475D3A20436F6D6D616E64206365
:100164006F6D706C65746564207375636365737318
:1001740066756C6C79207769746820636F64652098
:100184002230222E0A005B4C4F475D3A20496E769E
:10019400616C696420636F6D6D616E64206E616D66
:1001A40065210A005B4C4F475D3A204C697374200B
:1001B4006F6620617661696C61626C6520636F6D46
:0B01C4006D616E64733A0A002E20008B
:1001CF0048656C6C6F20776F726C64210A006C65E8
:1001DF00645F746F67676C650068656C6C6F006C4B
:0401EF0069737400BC
:1001F4001F920F920FB60F9211240BB60F922F93EA
:100204003F934F935F936F937F938F939F93AF939A
:10021400BF93EF93FF9380912008803221F18A30BD
:1002240069F08D3001F1E091824091E09E0F90934E
:100234008240F0E0E259FF4B808315C08EE690E4E3
:100244000E94480110928240EEE6F0E40190002002
:10025400E9F73197AF014E56504460E070E08EE606
:1002640090E40E944902FF91EF91BF91AF919F9159
:100274008F917F916F915F914F913F912F910F904B
:0C0284000BBE0F900FBE0F901F9018953E
:10029000CF92DF92EF92FF920F931F93CF93DF9352
:1002A0007C0102E010E4C0E0D0E0B801C7010E9488
:1002B0003002892B91F486E18C9FF0018D9FF00D27
:1002C0001124E050F04C0190F081E02D099584E577
:1002D00091E80E94DF0180E00BC021960A5E1F4F6B
:1002E000C630D10511F78AE891E80E94DF0181E06C
:1002F000DF91CF911F910F91FF90EF90DF90CF9002
:0203000008955E
:10030200CF93DF93CDB7DEB76697CDBFDEBFFB01DC
:1003120001900020E9F73197E61BF70B759708F576
:1003220020918340253010F01092834089839A8374
:10033200CE0103960E945A02A091834081E08A0F67
:100342008093834086E1A89FD0011124A050B04C35
:1003520086E1FE01319601900D928A95E1F781E0E6
:1003620001C080E06696CDBFDEBFDF91CF910895D8
:100372000F931F93CF9388EA91E80E94DF0100E078
:1003820010E4C1E3F80180819181892B71F08C2FF7
:100392000E9452028CEC91E80E94DF01C801029691
:1003A2000E94DF018AE00E9452020A5E1F4FCF5F65
:0C03B200C63341F7CF911F910F910895C1
:1003BE00EF92FF920F931F93CF93DF938C017C01EB
:1003CE00C0E0D0E006C0F70181917F010E94520289
:1003DE002196F80101900020E9F73197E01BF10B0F
:1003EE00CE17DF0780F3DF91CF911F910F91FF9012
:0403FE00EF900895DF
:1004020080E4809341040E941A0278946DED71E8B1
:1004120087E692E00E94810168EE71E882E692E04E
:100422000E9481016EEE71E889EB91E00E948101E8
:02043200FFCFFA
:10043400E0E2F8E083E896E08087918783E08783B1
:10044400A0E4B4E081E011968C93119782E01296B7
:0C0454008C9380E8858380EC86830895FB
:10046000DC01FB019D912191921303C09111FACF00
:0C047000292F892F90E0821B910908952C
:10047C00EC010E9470020E946F02CE010E94710278
:06048C00CE010E946D028A
:10049200FC01480F591FE417F50711F06193FBCFD8
:0204A2000895BB
:1004A400E0E2F8E0948195FFFDCF8093220808955F
:1004B400FC01DB012D91BD0121932111FACF089597
:0A04C4008FEC91E80E94DF0108951B
:0804CE0080E4809347040895C7
:0404D6000C94000082
:0404DA000E94A800D4
:0204DE0008957F
:0204E00008957D
:0204E20008957B
:00000001FF
